:1000000015C100002FC100002DC100002BC1000050
:1000100029C1000027C1000025C1000023C1000044
:1000200021C100001FC100000C947A121BC1000006
:1000300019C1000017C1000015C1000013C1000064
:1000400011C1000087C700000DC100000BC10000F6
:1000500009C1000099C1000005C1000003C10000F2
:1000600001C10000FFC00000FDC00000FBC0000097
:10007000F9C00000F7C00000F5C00000F3C00000A8
:10008000F1C00000EFC00000EDC00000EBC00000B8
:10009000E9C00000E7C00000E5C00000E3C00000C8
:1000A000E1C00000DFC00000DDC000001803410017
:1000B0005600520049005300500020006D006B00B4
:1000C0004900490000000C03410054004D00450068
:1000D0004C0000000403090412011001FF0000108D
:1000E000EB03042100020102030109000A000A00D7
:1000F0000B000C000D000D000E000F001000100092
:100100001200130013001400160016001800190046
:100110001A001C001D001F002000220023002500E3
:10012000270029002B002E00300032003400370059
:100130003A003D004000430046004A004E00520095
:1001400055005A005E00630068006D00730078007F
:100150007E0084008B0091009900A000A900B100EE
:10016000B900C300CC00D600E100EC00F7000401A8
:1001700011011E012D013B014B015B016C017D0151
:100180009101A501BA01CF01E601FE01160231027B
:100190004C026A028802A802CA02ED021103380367
:1001A00060038B03B803E70318044B048104B9040C
:1001B000F50434057505B90501064E069D06EF06E2
:1001C0004807A30704086508D0084009B6092B0AA8
:1001D000AB0A300BC30B510CEE0C8F0D400EF60E1C
:1001E000AF0F681047111412F512ED13E214F01559
:1001F000F9161B185C19911AE51B251D831E032097
:10020000AB21302332250F27F128F82A1A2D492F48
:10021000A1311434A1364539173C1A3F34426045A8
:10022000DF48704C400041014243030011241FBECF
:10023000CFEFDAE0DEBFCDBF11E0A0E0B1E0E0EF4C
:10024000F8E202C005900D92A03AB107D9F721E07B
:10025000A0EAB1E001C01D92A33BB207E1F743D091
:100260000C947614CDCE9BB19F7B892B8BB90895CE
:1002700084B7877F84BF0FB6F894A89580916000FB
:10028000886180936000109260000FBE90E080E86B
:100290000FB6F89480936100909361000FBE569A58
:1002A0005E980C945D1280E4DECF80E4DCCF42E304
:1002B00060E882E00E94C011811102C080E401C0A8
:1002C00080E0D1CF8EB3843069F4D5D182E08093C1
:1002D000E9008091E80082FF05C080E4C4DF86D099
:1002E00080E0C1CF0895C4DF64D080E4BCDF78949F
:1002F000E9DF0E944314FCCF00C0F9011082292FCE
:1003000033272230310559F02330310579F021307F
:10031000310591F582E190E028ED30E031C082E0D6
:10032000808380E290E02EE131E02AC0992781307D
:100330009105C9F02CF4892BF9F4E4EDF0E018C034
:100340008230910599F00397B9F48091000190E013
:1003500022E330E030930F0120930E0122E020834E
:1003600020E031E00DC0E6ECF0E002C0ECEAF0E0A5
:10037000849190E09F0104C080E090E020E030E0B4
:10038000FA0131832083089578941F920F920FB65B
:100390000F9211248F938AB5882321F08AB581505A
:1003A0008ABD01C015BC8F910F900FBE0F901F909A
:1003B0001895EAE7F0E087EA80838098AEE7B0E03E
:1003C0008C9181608C9380E480937C00ABE7B0E0FB
:1003D0008C918F7D8C938081806480838BE987BD35
:1003E00082E084BD80936E002BD1E2C50F931F93F2
:1003F000CF93DF931F92CDB7DEB70091F10084E673
:100400008ABD85E085BD043109F4C3C0E8F50A3032
:1004100009F4A8C048F5043018F5023008F051C0BE
:10042000013009F0C5C08091E8008B778093E80027
:1004300082E08093E9008091EC0081608093EC0081
:100440000093F1001092F1008AE08093F10040E007
:1004500050E06AE070E085E991E00E94A50FCBC012
:10046000063009F459C0A4C0013109F48DC028F444
:10047000003109F09DC066D4C3C0023109F48CC0BC
:10048000033109F483C094C0093109F48AC060F4CF
:10049000063109F47EC008F479C0073109F481C03F
:1004A000083109F47BC084C00D3109F47DC008F423
:1004B00075C0003509F47AC0013509F079C0CFD78D
:1004C0009FC01091F100023011F46091F100809111
:1004D000E8008B778093E80082E08093E9008091C8
:1004E000EC0081608093EC000093F100812F698320
:1004F000D9D06981023039F481FF0CC01092F1002B
:10050000812FE0D078C080FF05C01092F100812FCC
:10051000D1D06FC080EC6DC040E050E064E070E08E
:1005200084EA91E00E9439108091E8008B778093F3
:10053000E80082E08093E9008091EC008160809384
:10054000EC008091A4019091A501A091A601B09129
:10055000A701B7FF03C081E08093A30186E08093E9
:10056000F1000FC08091E8008B778093E80082E073
:100570008093E9008091EC0081608093EC0000930F
:10058000F1001092F10037C064D43AC0802FDDD062
:1005900037C0802F05D234C090D432C0802F9ED275
:1005A0002FC0802FF5D22CC035D32AC088D728C0C1
:1005B0002091F3008091F20090E0922B803491051D
:1005C00041F48091E8008B778093E8000E94F1115C
:1005D000EFCF8091E8008B778093E80082E08093F2
:1005E000E9008091EC0081608093EC000093F100C1
:1005F00089EC8093F1008091E8008E778093E80089
:1006000015BC0E94F11182E08093E9008091EC001A
:100610008E7F8093EC000F90DF91CF911F910F910F
:100620000895EEE3F1E09081891741F0339691E06F
:10063000EC35F907C1F780E090E00895CF01089507
:10064000CF93DF9381E090E00E945C14D82F80E08C
:1006500090E00E945C14C82FDF3F21F08EE9E1DFBB
:10066000FC01D283CF3F21F088E9DBDFFC01C283AC
:10067000DF91CF91089584E9D4DFEAE7F0E02081AB
:1006800020612083409178005091790062E3649F5B
:100690009001659F300D1124232F26952695FC018E
:1006A00022830895BEDF009719F0FC01818108952F
:1006B00080E00895B6DF009719F0FC01828108956B
:1006C00080E008951F93CF93DF931F92CDB7DEB7DD
:1006D000182F6983A6DF6981009789F0FC01628386
:1006E0001E3919F481E090E004C0183941F480E02B
:1006F00090E00F90DF91CF911F910C9464140F90B4
:10070000DF91CF911F91089590915C01992331F071
:100710008EBD0DB407FEFDCF8EB50895B0C4909187
:100720005C01992329F08EBD0DB407FEFDCF08951D
:10073000A6C480915C01882331F01EBC0DB407FE75
:10074000FDCF8EB5089580E09AC44F925F926F926C
:100750007F928F929F92AF92BF92CF92DF92EF9251
:10076000FF920F931F93CF93DF93CDB7DEB7C9509E
:10077000D1400FB6F894DEBF0FBECDBF182F40E0BA
:1007800050E069E070E0CE0101960E94EF0F6A81AF
:1007900079817A836983613081E0780788F080917C
:1007A000E8008B778093E80082E08093E9008091F5
:1007B000EC0081608093EC001093F10080ECD1C0DC
:1007C00040E050E0CE010A960E94EF0F89819A81A5
:1007D0000A968F739927892B39F48091E8008B77DB
:1007E0008093E8000E94F1118091E8008B7780935C
:1007F000E80082E08093E9008091EC0081608093C2
:10080000EC00133111F4C88401C0C9847090A401B4
:100810006090A501FE013A964F01A12CB12CE12C6C
:10082000F12C88E0582E4424439489819A81A8169B
:10083000B90608F066C0F40101914F01DB80809198
:10084000A301882319F06ED41092A3018D8167DF74
:100850008091A50164DF8091A40161DF802F5FDFBB
:10086000133119F49D8195259D83E114F10479F4E8
:100870000C1569F08F81A0FE04C0133111F488605B
:1008800001C0877F8F83E090A401F090A501D0FC88
:1008900013C0E114F10431F4D3FC04C08D2D897F21
:1008A0008260D82E0F812C814C2DB7018D2D43D421
:1008B000811128C0E12CF12CA0FC02C01531E9F413
:1008C0008091A4019091A501A091A601B091A701EA
:1008D0000196A11DB11D8093A4019093A501A09341
:1008E000A601B093A701133141F4AA27BB27892B96
:1008F0008A2B8B2B11F44092A301FFEFAF1ABF0A92
:1009000094CF80E09B8197FF2AC08E8108DF862DDF
:1009100006DF872D04DF80E002DF8B8185FF06C0C4
:10092000E114F10419F48F7C80618B830F812C8199
:100930004C2DB7018B81FFD3133189F44091A40171
:100940005091A5016091A6017091A70166277727B4
:10095000452B462B472B19F491E09093A30110935C
:10096000F1008093F1008091E8008E778093E80099
:10097000C75FDE4F0FB6F894DEBF0FBECDBFDF916D
:10098000CF911F910F91FF90EF90DF90CF90BF908C
:10099000AF909F908F907F906F905F904F90089551
:1009A000DF92EF92FF920F931F93CF93DF9300D0CC
:1009B0001F92CDB7DEB7F82E40E050E063E070E064
:1009C000CE0101960E94EF0F89819A8199838A83D3
:1009D0008091E8008B778093E80082E08093E900C3
:1009E0008091EC0081608093EC00F092F100109215
:1009F000F10000E010E088E0E82EDD24D394898146
:100A00009A810817190708F04AC08091A30188232A
:100A100019F088D31092A3018B8181DE8091A5010A
:100A20007EDE8091A4017BDE84DE8093F1008091E4
:100A3000E80085FD07C08091E8008E778093E8008C
:100A40000E94F11184E1F81203C08B818E258B8303
:100A500000FD03C086E1F8121FC04091A40150912F
:100A6000A5016091A6017091A7014F5F5F4F6F4F85
:100A70007F4F4093A4015093A5016093A60170930A
:100A8000A70186E1F81641F066277727452B462B0C
:100A9000472B11F4D092A3010F5F1F4FB0CF1092DC
:100AA000F1009091E8008091E8008E778093E80053
:100AB00095FD09C00E94F1118091E8008E77809326
:100AC000E8000E94F1110F900F900F90DF91CF91ED
:100AD0001F910F91FF90EF90DF900895CF92DF92DA
:100AE000EF92FF920F931F93CF93DF93CDB7DEB7B3
:100AF00029970FB6F894DEBF0FBECDBFD82E40E0C9
:100B000050E065E070E0CE0101960E94EF0F9091F9
:100B1000E8009B779093E80082E08093E900909151
:100B2000EC0091609093EC007E0182E0E80EF11CF5
:100B30008E010A5F1F4F84E0C82EC00EF70181911D
:100B40007F01E2DDF80181938F01CE12F7CFD092C1
:100B5000F1001092F1008981FE01E80FF11D8581FD
:100B60008093F1001092F1008091E8008E778093DD
:100B7000E80029960FB6F894DEBF0FBECDBFDF9117
:100B8000CF911F910F91FF90EF90DF90CF9008953C
:100B9000EF92FF920F931F93CF93DF9300D000D07B
:100BA000CDB7DEB7F82E40E050E064E070E0CE0153
:100BB00001960E94EF0F9091E8009B779093E800D8
:100BC00082E08093E9009091EC0091609093EC00BA
:100BD0008E010F5F1F4F84E0E82EE00EF801819137
:100BE0008F019DDDE012FACFF092F1001092F1003A
:100BF0001092F1008091E8008E778093E8000F90CA
:100C00000F900F900F90DF91CF911F910F91FF9058
:100C1000EF900895FF920F931F93CF93DF93CDB77B
:100C2000DEB7C250D1400FB6F894DEBF0FBECDBFC5
:100C300040E050E063E070E0CE0101960E94EF0FCB
:100C4000698170E040E050E0CE0104960E94EF0F11
:100C50008091E8008B778093E80082E08093E90040
:100C60008091EC0081608093EC008DE18093F10035
:100C70001092F10010E08B81181778F48981181711
:100C800040F4E4E0F0E0EC0FFD1FE10FF11D808186
:100C900001C080E044DD1F5FEECF00E08A810817CD
:100CA00010F58981181778F4FF24F394F10EE4E02D
:100CB000F0E0EC0FFD1FE10FF11D808125DD809339
:100CC000F1001F2D03C035DD8093F1008091E80015
:100CD00085FD07C08091E8008E778093E8000E9430
:100CE000F1110F5FDBCF1092F1009091E80080913D
:100CF000E8008E778093E80095FD09C00E94F1110D
:100D00008091E8008E778093E8000E94F111CE5F19
:100D1000DE4F0FB6F894DEBF0FBECDBFDF91CF918F
:100D20001F910F91FF900895882359F09AB5815033
:100D3000992339F0EFE9FFE03197F1F700C00000A7
:100D4000F3CF0895BF92CF92DF92EF92FF920F936D
:100D50001F93CF93DF93CDB7DEB72F970FB6F894DD
:100D6000DEBF0FBECDBF40E050E06BE070E0CE01D3
:100D700001960E94EF0F8091E8008B778093E80046
:100D800082E08093E9008091EC0081608093EC0028
:100D90001092A4011092A5011092A6011092A70131
:100DA0008B81C2DF45D181E093D18A81BDDF7E0195
:100DB0008CE0E80EF11C84E0B82EBE0C8C819FEF15
:100DC000980F9C83882351F18AB5882339F1CE018D
:100DD00008966C0187018D81A7DFF60181916F0173
:100DE00093DCF80181938F01BE12F5CF8F818823A8
:100DF00051F0EBE0F0E0EC0FFD1FE80FF11D9081EA
:100E00008E81981302C080E00AC080E061D18A819F
:100E10008BDF81E05DD18A8187DFD0CF80EC90E1EC
:100E20009093F1008093F1008091E8008E77809399
:100E3000E8002F960FB6F894DEBF0FBECDBFDF914E
:100E4000CF911F910F91FF90EF90DF90CF90BF90C7
:100E500008950F931F93CF93DF9300D0CDB7DEB7E4
:100E600040E050E062E070E0CE0101960E94EF0F9A
:100E700008EE10E0F80180818B77808382E0809318
:100E8000E900ECEEF0E080818160808389814CDFB5
:100E900080E01ED1A1D08A8147DFE1EFF0E081E15F
:100EA00080831082F80180818E7780830F900F906D
:100EB000DF91CF911F910F910895EF92FF920F93C1
:100EC0001F93CF93DF9300D000D000D0CDB7DEB713
:100ED00040E050E066E070E0CE0101960E94EF0F26
:100EE0008091E8008B778093E80082E08093E900AE
:100EF0008091EC0081608093EC008E010D5F1F4FAC
:100F00007E0187E0E80EF11CF80181918F0107DC7A
:100F10000E151F05C9F78A81811104C0898104DF7C
:100F200080E001C0E1D092E19093F1008093F10064
:100F30008091E8008E778093E80026960FB6F894AB
:100F4000DEBF0FBECDBFDF91CF911F910F91FF90FC
:100F5000EF9008951F920F920FB60F9211248F9366
:100F6000199908C08091A10187FF02C02A9A19C06F
:100F70002A9817C08091A101880F8093A1018091C8
:100F8000A00181508093A001811104C010928100C2
:100F900082E086BB1B9B05C08091A101816080938C
:100FA000A101199A8F910F900FBE0F901F90189565
:100FB000259A10926F00109285001092840081E0B3
:100FC00090E0909389008093880080E48093800073
:100FD00089E080938100089580915C01882349F025
:100FE00084B1897F84B985B1867F85B91CBC1DBC5D
:100FF000089584B1897F84B985B1867F85B9D8CFBA
:1010000092E090936F001092850010928400E82F78
:10101000F0E0EE0FFF1FE452FF4F85919491909303
:1010200089008093880010928000109281000895BA
:1010300088E940DB8730D0F491E090935C01E82FA1
:10104000F0E0EC5DFD4FE491209A289A84B186602F
:1010500084B923982B9A8DB5E6FF02C0816001C048
:101060008E7F8DBD2098E065ECBD089510925C01E7
:1010700094B1966094B995B1996095B9C1CF8093B8
:10108000A10188E08093A0018091A10187FF02C0A7
:101090002A9A01C02A9810928500109284008AE052
:1010A000809381008091A001882319F08AB5811175
:1010B000F9CF109281008091A101089590915C0177
:1010C000992329F08EBD0DB407FEFDCF0895D7CF2B
:1010D000882339F0279A8EE9EDDA811103C02F9A1F
:1010E000089527982F98089580EFE8DF80E0E6DFE5
:1010F00080E0E4DF80915C01882331F01EBC0DB4F8
:1011000007FEFDCF8EB502C080E0B9DF80FF03C0CF
:101110008AB58111E9CF8AB5811102C081E80895AD
:1011200080E008958DE4CADF80E0C8DF8091A601E9
:10113000C5DF80E0C3CF0F931F93CF93DF93D62FEC
:10114000172FC42F8E77E82FF0E0E830F10579F102
:1011500034F4E230F10559F03497A9F02AC0E032B6
:10116000F10589F0E034F10511F1709711F5822F46
:10117000DBDD1FC00DB407FEFDCF8EB58C1312C092
:101180009AB5992379F0802F99DF812F97DF8D2FE2
:1011900095DF80915C01882311F01EBCEBCF80E0CD
:1011A0006EDFECCF8AB5811104C080E803C09CDFFC
:1011B00001C080E094E69ABDDF91CF911F910F911D
:1011C0000895AF92BF92CF92DF92EF92FF920F936A
:1011D0001F93CF93DF93CDB7DEB7C850D1400FB682
:1011E000F894DEBF0FBECDBF40E050E068E070E095
:1011F000CE010196F4D68B819C812D813E813B836B
:101200002C839D838E837F8168856F83788740E000
:1012100050E0CE010996E3D68F81988509968F73A9
:101220009927892B39F48091E8008B778093E80027
:101230000E94F1118091E8008B778093E80082E0B2
:101240008093E9008091EC0081608093EC008091B4
:10125000A20181112DC0298121504B815C816D81BA
:101260007E812630A0F430E0F901E958FE4F8081FC
:10127000F901EF58FE4F9081F901E559FE4FE081E9
:10128000D901AB59BE4F2C912223D9F003C0E6E21D
:1012900093E28EE2AF80B8849E01275F3F4F6901E1
:1012A0007A018B012A81482F6E2F892F51D40BC0D0
:1012B0004F815885BE01675F7F4F8B819C81ECD544
:1012C00002C0298516D4882311F080E001C083E094
:1012D00090E59093F10094E09093F1008093F100F9
:1012E0008091E8008E778093E800C85FDE4F0FB6EC
:1012F000F894DEBF0FBECDBFDF91CF911F910F914C
:10130000FF90EF90DF90CF90BF90AF900895CF9374
:10131000DF93CDB7DEB7C750D1400FB6F894DEBF2C
:101320000FBECDBF40E050E067E070E0CE018F5FC0
:101330009E4F55D6CE5FDE4F8881C250D140CD5FE3
:10134000DE4F9881C350D140CC5FDE4F2881C4501E
:10135000D140CB5FDE4F3881C550D140CE5FDE4FEC
:101360003883C250D140CD5FDE4F2883C350D14077
:10137000CC5FDE4F9883C450D140CB5FDE4F888373
:10138000C550D140CA5FDE4F8881C650D140C95F89
:10139000DE4F9881C750D140CA5FDE4F9883C65058
:1013A000D140C95FDE4F8883C750D1408091E800AB
:1013B0008B778093E80082E08093E9008091EC00D5
:1013C00081608093EC008091A201CA5FDE4F28818A
:1013D0003981C650D140811112C0CE5FDE4F688185
:1013E00079818A819B81C250D140AE014F5F5F4FAE
:1013F0003CD3882311F080E00EC083E00CC0A9012B
:10140000BE016F5F7F4FCE5FDE4F88819981C250F2
:10141000D14015D5EECF90E59093F10095E09093F3
:10142000F1008093F10081110BC0CA5FDE4F68812B
:101430007981C650D14040E050E0CE01019685D57B
:101440008091E8008E778093E800C95FDE4F0FB689
:10145000F894DEBF0FBECDBFDF91CF910895CF933B
:10146000DF931F92CDB7DEB740E050E061E070E05F
:10147000CE010196B4D58091E8008B778093E80087
:1014800082E08093E9008091EC0081608093EC0021
:1014900089818093A20181E58093F1008981813067
:1014A00011F480EC01C080E08093F1008091E800AD
:1014B0008E778093E8000F90DF91CF910895CF93BE
:1014C000DF9300D000D000D0CDB7DEB78091F1001F
:1014D000843009F492C038F4823081F108F04AC0B7
:1014E000813051F029C1863009F48BC008F487C0DF
:1014F000873009F4CFC020C18091E8008B778093BA
:10150000E80082E08093E9008091EC0081608093A4
:10151000EC008091A201811102C022D205C082306C
:1015200011F447D401C080E090E59093F10091E080
:101530009093F10098279093F100F9C09091E80002
:101540009B779093E8008093E9008091EC008160A4
:101550008093EC008091A201811102C040D201C0B1
:1015600063D480E58093F10082E08093F1001092D3
:10157000F100DDC040E050E065E070E0CE01019692
:101580002ED58A819B812C813D813A832B839C833C
:101590008D838091E8008B778093E80082E08093D0
:1015A000E9008091EC0081608093EC008091A201C1
:1015B000E981811114C0E150E83028F4F0E0E358EB
:1015C000FE4F808101C080E04A815B816C817D811A
:1015D00031D3882311F080E00BC083E009C0E130F3
:1015E00011F084E101C080E16A817B8191D4F1CF67
:1015F00090E59093F10093E096C0E3DD9DC087DE17
:101600009BC040E050E061E070E0CE010696E7D478
:101610008091E8008B778093E80082E08093E90076
:101620008091EC0081608093EC008091A201811197
:1016300012C08E81813031F0823011F489E303C011
:1016400088E701C088E3BE016F5F7F4FD3D181116E
:1016500004C083E003C081E001C080E090E5909386
:10166000F10096E09093F1008093F10081115FC04A
:1016700089819A81AB81BC81CD01AA27BB27809348
:10168000F10089819A81AB81BC818093F100892F1F
:1016900099274BC08091F100833041F168F481308B
:1016A000A1F0823071F58091F1009091F10090935A
:1016B0005F018093600123C08430E9F0853009F533
:1016C0008091F1008091F1001AC08091F100909119
:1016D000F1002091F1003091F100309361012093ED
:1016E0006201909363018093640109C08091F100CD
:1016F00080935E0104C08091F10080935D0180E0E1
:1017000001C081E09091E8009B779093E80092E01F
:101710009093E9009091EC0091609093EC0090E53B
:101720009093F10097E09093F1008093F100809105
:10173000E8008E778093E80026960FB6F894DEBF17
:101740000FBECDBFDF91CF9108954D99FECF4D9B38
:10175000FECF4D99FECF5B9A539A8091C9008F7E40
:101760008093C9008091C90088608093C90081E09E
:101770008093A80108958091C80086FFFCCF8091D6
:10178000C80080648093C8008091C900877F8093DF
:10179000C9008091C90080618093C90053985B980B
:1017A0001092A80108958091A8018111E4DF80ECD6
:1017B0008093C8001092C9001092CA008AB1877D38
:1017C0008AB98BB1837D8BB908958091A80181116D
:1017D000D2DF8091C800806C8093C8001092C9004D
:1017E0001092CA008AB1877D8AB98BB1837D8BB98B
:1017F00027982F980895CF93DF931F92CDB7DEB728
:101800009091A801911103C089839FDF89819091F4
:10181000C80095FFFCCF9091C80090649093C800D9
:101820008093CE000F90DF91CF9108958091A80111
:101830008111A1DF8091C80087FD03C08AB58111A5
:10184000F9CF8091CE0008958091A801811101C047
:101850007CDF8CE04D99FECF4D9BFECF4D99FECFA6
:101860008150C1F708951092A8018AB188628AB99F
:1018700052985B9A8FE891E00197F1F700C0000061
:1018800083E090E09093CD008093CC0088E080933B
:10189000C9008FE68093CA00D7DFD6CF1092A80187
:1018A000279A2F988FE891E00197F1F700C0000088
:1018B0008AB188628AB9529883E090E09093CD0013
:1018C0008093CC0088E08093C9008FE68093CA00A3
:1018D000BBDFBACF1F93CF93DF9300D0CDB7DEB776
:1018E000182F862F79839A8386DF7981872F83DF6C
:1018F000812F81DF9A81892F0F900F90DF91CF91F7
:101900001F9179CF0F931F93409161015091620114
:1019100060916301709164018A019B01082BC901E8
:10192000B8011F910F91D6CF80E865DF7FDF9AB5B0
:10193000992321F081FFF8CF81E0089580E0089598
:101940008BE659DF8FE0DEDF80E255DF6FDF9AB58F
:10195000992321F087FDF8CF81E0089580E0089574
:10196000DF92EF92FF920F931F93CF93DF93CDB748
:10197000DEB728970FB6F894DEBF0FBECDBF73DF7A
:1019800081EC39DF89E537DF82EC35DF82E033DF58
:1019900080EE31DF8E01075F1F4FCE0101967C0183
:1019A00088E0D82EE5E8F1E0D7018D2D01900D9269
:1019B0008A95E1F7F80182918F011DDF0E151F0551
:1019C00089F728960FB6F894DEBF0FBECDBFDF9122
:1019D000CF911F910F91FF90EF90DF90A5CFA4DFE3
:1019E00081EC09DF80E007DF81E805DF1FDF81117F
:1019F000F7CFD9CE0F931F93CF93DF93182FEB011F
:101A0000188219821A821B829BDF882341F18CE4A1
:101A1000F2DE8AE077DF812FEEDE8CE4ECDE8BE015
:101A200071DF81E0E8DE80DF8823C9F089DF882369
:101A3000B1F08BE6E0DE84E065DF80EADCDE82E0A8
:101A4000DADE84E2D8DE8E010D5F1F4FEFDE899370
:101A5000C017D107D9F79AB581E0911101C080E094
:101A6000DF91CF911F910F910895CF92DF92EF9266
:101A7000FF920F931F93CF93DF936B017C01EA01D9
:101A800089015EDF882361F18CE4B5DE8AE03ADF0C
:101A900083E4B1DE02301105B8F08BE6ACDEC7019D
:101AA000B60118DF80EAA7DE8FEF800FA4DE84E2A4
:101AB000A2DE0C0F1D1FC017D10769F08AB588235D
:101AC00051F0B4DE8993F7CF8CE095DEC701B60103
:101AD00001DFACDE88839AB581E0911101C080E01E
:101AE000DF91CF911F910F91FF90EF90DF90CF90FA
:101AF0000895FF920F931F93CF93DF9300D000D0F0
:101B0000CDB7DEB7182FF22E49835A836B837C83BF
:101B100017DF082F882389F08CE46DDE8AE0F2DE7F
:101B2000812F69DE8CE467DE49815A816B817C817B
:101B3000CB01BA01CFDE8F2D5EDE802F0F900F908C
:101B40000F900F90DF91CF911F910F91FF9008950B
:101B50004F925F926F927F928F929F92AF92BF92BD
:101B6000CF92DF92EF92FF920F931F93CF93DF9369
:101B7000C82FD62F842E922E2701380120FF11C0A6
:101B8000DFDE811102C0C0E043C08CE434DE8AE0B5
:101B9000B9DE8D2F30DE8CE42EDE8BE0B3DE81E00B
:101BA0002ADEA114B10421F491FC20C0C1E030C0B0
:101BB000C7DE882341F38CE41EDE8AE0A3DE8C2F8F
:101BC0001ADE8BE618DEC301B20184DE80EA13DE82
:101BD0008FEF8A0D10DE84E60EDEE601AC0CBD1C34
:101BE000CA15DB0509F3899106DEFACFA9DEC82FF5
:101BF000882309F4C8CF8CE4FEDD8AE083DE882DDB
:101C0000FADD8CE4F8DDC301B20164DE80E0F3DDCF
:101C10008C2FDF91CF911F910F91FF90EF90DF906C
:101C2000CF90BF90AF909F908F907F906F905F907C
:101C30004F9008951F93CF93DF9300D000D0CDB77E
:101C4000DEB7182F49835A836B837C8379DE498101
:101C50005A816B817C81882309F467C08CE410343D
:101C600029F4C9DD8AE04EDE80E440C049835A830E
:101C70006B837C83103309F040C0BDDD8AE042DE17
:101C800086E3B9DD8CE4B7DD8BE03CDE81E0B3DDDB
:101C900057DE882309F449C08CE4ADDD8AE032DEEA
:101CA00083E3A9DD8BE6A7DD49815A816B817C81C5
:101CB000CB01BA010FDE80EA9EDD80915F01815089
:101CC0009ADD84E698DD10E0812F90E020915F019D
:101CD000309160018217930720F480E08CDD1F5F54
:101CE000F3CF8CE488DD8AE00DDE80E384DD8CE4D4
:101CF00082DD8BE007DE81E00FC07DDD8AE002DE61
:101D0000812F79DD8CE477DD49815A816B817C817B
:101D1000CB01BA01DFDD80E06EDD0F900F900F90F8
:101D20000F90DF91CF911F91FFCD80E00F900F902A
:101D30000F900F90DF91CF911F910895982F9F7072
:101D400090698073880F892B56CD1F93CF93DF93B3
:101D50001F92CDB7DEB7182F88E699834CDD812F0F
:101D60004ADD89E648DD9981892F0F90DF91CF9177
:101D70001F9141CD80E83FDD59DD9AB5992321F0CF
:101D800081FFF8CF81E0089580E0089590915D0192
:101D9000892F8F7080619073990F892B2CDD46DD20
:101DA0009AB5992321F087FDF1CF81E0089580E075
:101DB0000895DF92EF92FF920F931F93CF93DF93DB
:101DC000CDB7DEB728970FB6F894DEBF0FBECDBFF4
:101DD00065DD82EC10DD82E00EDD80EE0CDD8E0133
:101DE000075F1F4FCE0101967C0188E0D82EEDE8F9
:101DF000F1E0D7018D2D01900D928A95E1F7F80160
:101E000082918F01F8DC0E151F0589F728960FB611
:101E1000F894DEBF0FBECDBFDF91CF911F910F9120
:101E2000FF90EF90DF90A6CFA5DF80ECE4DC80E0B0
:101E3000E2DC80E8E0DCFADC8111F7CFC6CCEF927F
:101E4000FF920F931F93CF93DF93EC017B018A01E5
:101E50009DDF8823D1F080915E0170DF80E0CBDCD4
:101E6000CE0173DFE7010E0D1F1DC017D10741F032
:101E70008AB5882329F084E2BEDCD8DC8993F5CFCB
:101E80009AB581E0911101C080E0DF91CF911F915F
:101E90000F91FF90EF900895CF92DF92FF920F93F2
:101EA0001F93CF93DF936C018B01EA016FDFF82E54
:101EB000811102C0F12C23C0C0FF06C0F801EC0F55
:101EC000FD1F8FEF8083219680915E0137DF8DE1CA
:101ED00092DCC6013ADF209791F058DF882351F356
:101EE00084E689DCF801808186DC84E684DC0E5F90
:101EF0001F4FF801319780817EDC2297ECCF8F2D28
:101F0000DF91CF911F910F91FF90DF90CF900895B7
:101F10001F93CF93DF93182FEB0138DF882381F0D5
:101F200080915E010BDF812F66DCCE0181600DDFC9
:101F300080E661DC80E05FDCDF91CF911F9126CFEE
:101F400080E0DF91CF911F910895CF92DF92EF92C1
:101F5000FF920F931F93CF93DF93EC018B017A01D4
:101F600040D2811133C0E114F10439F0F7018081CE
:101F70009181081B190BC80FD91FC12CD12C011539
:101F8000110519F18091E80085FD16C08091E800E7
:101F90008E778093E80077D4E114F10449F0F701DB
:101FA00080819181C80ED91ED182C08285E00EC089
:101FB00018D2882321F30AC089918093F10001503F
:101FC0001109FFEFCF1ADF0ADACF80E0DF91CF915E
:101FD0001F910F91FF90EF90DF90CF900895CF92D7
:101FE000DF92EF92FF920F931F93CF93DF93EC0159
:101FF0008B017A01F6D1811133C0E114F10439F07B
:10200000F70180819181081B190BC80FD91FC12CC2
:10201000D12C0115110519F18091E80085FD16C03C
:102020008091E8008B778093E8002DD4E114F104CF
:1020300049F0F70180819181C80ED91ED182C082FA
:1020400085E00EC0CED1882321F30AC08091F10033
:10205000899301501109FFEFCF1ADF0ADACF80E030
:10206000DF91CF911F910F91FF90EF90DF90CF9074
:102070000895CF92DF92EF92FF920F931F93CF9329
:10208000DF93EC018B017A01ACD1811139C0980149
:1020900021503109C20FD31FE114F10439F0F701C7
:1020A00080819181081B190BC81BD90BC12CD12C25
:1020B0000115110521F18091E80085FD16C0809180
:1020C000E8008B778093E800DED3E114F10449F057
:1020D000F70180819181C80ED91ED182C08285E02E
:1020E0000FC07FD1882321F30BC08091F10088833A
:1020F000219701501109FFEFCF1ADF0AD9CF80E0F5
:10210000DF91CF911F910F91FF90EF90DF90CF90D3
:1021100008952091B1013091B2012617370748F098
:102120006115710539F42091E8002E772093E800BD
:1021300001C0B90140E061157105A1F12EB3222360
:1021400009F442C0253009F441C02091E80023FD84
:102150003FC02091E80022FD31C02091E80020FF1F
:10216000EACF4091F3002091F20030E0342BFC01E3
:10217000CF016115710559F02031310540F481918D
:102180008093F100615071092F5F3F4FF1CF41E023
:102190002031310509F040E02091E8002E772093AE
:1021A000E800C9CF4111CACF09C08EB3882361F0BE
:1021B000853061F08091E80083FD0AC08091E800DD
:1021C00082FFF3CF80E0089582E0089583E00895D0
:1021D00081E008952091B1013091B20126173707AF
:1021E00048F06115710539F42091E8002E772093AD
:1021F000E80001C0B901FC0120E06115710589F119
:102200008EB3882309F43FC0853009F43EC0809125
:10221000E80083FD3CC08091E80082FD2EC08091E3
:10222000E80080FFEACF2091F3008091F20090E077
:10223000922B6115710559F08031910540F424917C
:102240002093F1003196615071090196F2CF21E09F
:10225000409709F020E08091E8008E778093E800B5
:10226000CCCF2111CDCF09C08EB3882361F085304A
:1022700061F08091E80083FD0AC08091E80082FF50
:10228000F3CF80E0089582E0089583E0089581E02F
:102290000895CF92DF92EF92FF920F931F93CF9307
:1022A000DF93EB012091B1013091B201261737077E
:1022B00040F0209739F42091E8002E772093E80031
:1022C00001C0E9017C0180E02097D1F19EB3992300
:1022D00009F448C0953009F447C09091E80093FD97
:1022E00045C09091E80092FD37C09091E80090FFC2
:1022F000EBCF8091F3000091F20010E0182B680101
:10230000C601801B910B8E0D9F1D209761F020E16F
:10231000C216D10440F4D0D28093F10021972FEF60
:10232000C21AD20AEDCF7C0181E090E1C916D10436
:1023300009F080E09091E8009E779093E800C4CF88
:102340008111C4CF09C08EB3882361F0853061F05C
:102350008091E80083FD0AC08091E80082FFF3CFFE
:1023600080E005C082E003C083E001C081E0DF912E
:10237000CF911F910F91FF90EF90DF90CF90089534
:102380008F708093E900EBEEF0E0808181608083C4
:10239000EDEEF0E010826093EC0040838091EE005F
:1023A000881F8827881F08958091AB0187FF0FC081
:1023B0008091E80082FD04C08EB38111F9CF10C076
:1023C0008091E8008B770AC08EB3882349F0809112
:1023D000E80080FFF9CF8091E8008E778093E800D5
:1023E00008952091E4003091E50095E64091EC00DD
:1023F000842F817040FF21C08091E80080FD1BC0C8
:102400008EB3882391F0853091F08091EB0085FDAB
:1024100010C04091E4005091E5004217530731F39A
:102420009A01915019F784E0089582E0089583E0BD
:10243000089581E0089580E008954091E80042FF0A
:10244000DFCF08950F931F93CF93DF9346D04DD0E6
:10245000C8EDD0E088818F77888388818068888301
:1024600088818F7D888319BC1EBA1092A90100EE65
:1024700010E0F80180818B7F808388818160888370
:1024800042E160E080E07CDFE1EEF0E080818E7F81
:102490008083E2EEF0E080818160808380818860CB
:1024A0008083F80180818E7F80838881806188832A
:1024B000DF91CF911F910F910895E8EDF0E08081B9
:1024C0008F7E8083E7EDF0E080818160808384E00F
:1024D00082BF81E08093AA01B5CFE8EDF0E0808172
:1024E0008E7F80831092E20008951092DA0010929D
:1024F000E10008951F920F920FB60F9211242F93AF
:102500003F934F935F936F937F938F939F93AF937B
:10251000BF93EF93FF938091DA0080FF1DC08091FD
:10252000D80080FF19C08091DA008E7F8093DA0096
:102530008091D90080FF0CC080E189BD82E189BD16
:1025400009B400FEFDCF81E08EBB0E94530104C0A0
:1025500019BC1EBA0E9455018091E10080FF17C08E
:102560008091E20080FF13C08091E2008E7F809313
:10257000E2008091E20080618093E2008091D800C7
:1025800080628093D80019BC85E08EBB7BD180919E
:10259000E10084FF2EC08091E20084FF2AC080E128
:1025A00089BD82E189BD09B400FEFDCF8091D800CC
:1025B0008F7D8093D8008091E1008F7E8093E10031
:1025C0008091E2008F7E8093E2008091E200816042
:1025D0008093E2008091A901882311F084E007C074
:1025E0008091E30087FD02C081E001C083E08EBBE3
:1025F00049D18091E10083FF21C08091E20083FFF7
:102600001DC08091E100877F8093E10082E08EBB56
:102610001092A9018091E1008E7F8093E10080916A
:10262000E2008E7F8093E2008091E20080618093DF
:10263000E20042E160E080E0A3DE24D1FF91EF916F
:10264000BF91AF919F918F917F916F915F914F91CA
:102650003F912F910F900FBE0F901F9018951F93D1
:10266000CF93DF9300D01F92CDB7DEB7EBEAF1E056
:1026700088E08E0F9091F10091938E13FBCF02D1E1
:102680008091E80083FFE9C08091AB019091AC019B
:10269000953009F466C030F4913059F168F0933008
:1026A00041F1DBC0983009F4AAC0993009F4B9C0EF
:1026B000963009F0D2C076C0803881F0823809F0B7
:1026C000CCC08091AF018F708093E9008091EB00C6
:1026D00085FB882780F91092E90001C080E0909185
:1026E000E800977F9093E8008093F1001092F1004A
:1026F00091C0282F2D7F09F0B0C0823009F0ADC005
:102700008091AD01811127C08091AF018F7009F4D4
:10271000A4C08093E9002091EB0020FF1CC09330FF
:1027200021F48091EB00806214C09091EB009061E5
:102730009093EB0021E030E0A90102C0440F551F47
:102740008A95E2F74093EA001092EA008091EB004C
:1027500088608093EB001092E9008091E800877F09
:102760005CC081117AC01091AD011F778091E300A8
:102770008078812B8093E3008091E800877F8093AD
:10278000E80012DE8091E80080FFFCCF8091E3003A
:1027900080688093E300111102C082E001C083E0F1
:1027A0008EBB5BC08058823008F057C09E012D5F01
:1027B0003F4FAE014F5F5F4F6091AF018091AD0120
:1027C0009091AE010E947C01BC01892B09F445C0A7
:1027D0008091E800877F8093E8002B8189819A812E
:1027E000211102C0F7DC05C0213011F452DD01C017
:1027F00090DC8091E8008B778093E8002EC08038D1
:1028000061F58091E800877F8093E8008091A901BD
:102810008093F1008091E8008E778093E800C4DD1A
:102820001CC081111AC09091AD019230B0F480911A
:10283000E800877F8093E8009093A901B5DD80913F
:10284000A901811106C08091E30087FD02C081E0EB
:1028500001C084E08EBB0E9457018091E80083FF95
:102860000AC08091E800877F8093E8008091EB00A8
:1028700080628093EB000F900F900F90DF91CF91CB
:102880001F9108950895CF938EB3882399F0C09136
:10289000E900CF709091EC00892F817090FD80E865
:1028A000C82B1092E9008091E80083FDD8DECF703C
:1028B000C093E900CF910895F999FECF92BD81BDF3
:1028C000F89A992780B50895262FF999FECF92BDE1
:1028D00081BDF89A019700B4021639F01FBA20BDE5
:1028E0000FB6F894FA9AF99A0FBE0895F894FFCFAC
:1028F0001C03300030003000320030003000300067
:1029000031003200330034003500000000000902BD
:102910002000010100C0320904000002FF00000095
:102920000705820240000A0705020240000A8001F2
:102930000081010090010091010192011894012190
:102940009803069E0301A10100A403000132332075
:1029500000C00100010101010000012626362626E3
:1029600026232333232323242C354C081A402068A4
:1029700030222A32181289AB45CDD888FF1289AB94
:1029800045CDD888FF4156524953505F4D4B3200D8
:00000001FF
